:020000020000FC
:10000000B7CDAEC10000000020C000008EC00000CF
:10001000000098C000000000000000000203040679
:10002000080C10182030406080000406080C1018DE
:100030002030406080A0C0000003070F1F000D0D9E
:1000400004050D050305030302004FB662FD0CC055
:10005000552041F00994C52DC095089483FDC7959E
:10006000C4BD64604FBE1895C0916400089483FDC0
:10007000C795C4BD6B7FC0916400CF3F09F41EC01B
:1000800070FF1AC082FD05C04FBE9798AC98959836
:10009000189576FD0EC064FD0CC0C091B100C0FD86
:1000A000AB98C1FDAD98C2FD9498CAEFC095CA95B2
:1000B000F1F79798AC9895984FBE189524BCCC272B
:1000C000C064C8BF6460F8CFC6CF70FFC4CF64FD02
:1000D000C2CF979AC0CF70FFBECF64FDBCCFAC9AA1
:1000E000BACF70FFB8CF64FDB6CF959AB4CFAB9AB4
:1000F00070FFB1CF64FDAFCFC7E0CA95F1F7979A13
:10010000AACFAD9A70FFA7CF64FDA5CFC7E0CA956F
:10011000F1F7AC9AA0CF949A70FF9DCF64FD9BCF6E
:10012000C7E0CA95F1F7959A96CF4FB6C9B7CF7E7B
:10013000C9BF6E7FCCB5CE0DDDB5DF1DDBBDCABD41
:100140004FBE18953FB68F7EABB7A074A2118061E9
:10015000A0E0ABBFA9B7AE7FA9BF7894A09168001B
:10016000AA2341F085FD2EC0A0916800AA95A09316
:10017000680028C040E050E085FD14C0A0B396FDA3
:10018000A095A2FD4FEFA3E096FDA2E0A5BFAA2790
:10019000A064AABF8D7FA0B396FDA095A2FD5FEFDE
:1001A000451741F7A8E161FDA093680085FD03C0F4
:1001B000A8E1A0936800409396008160442311F069
:1001C0002092990085FD0EC0A0916900AA2331F00C
:1001D000A0916900AA95A093690004C08061AA2734
:1001E000A064AABF80FF3CC0A09196004A2F61FF87
:1001F0008E7F85FD1CC0A091B400A430C1F4403FA7
:1002000008F040EFA42FA295AF704A0F5091B600AE
:10021000533069F0A695A69550FD01C0A69552FDF4
:1002200003C0A41B4A2F03C04A0F08F44FEF4093AA
:100230006100A72FA670A1F073FD12C0A0917000FD
:10024000AA0FAA0F50919E0056955695541708F084
:10025000452F4A0F4093610018F4AFEFA09361005F
:100260004091B400443009F03EC0A0916100A093D9
:10027000630040916300A0919B004A1708F04A2F49
:10028000A0919D004A1708F04A2F542EA091A0007B
:10029000AA2309F422C0542F5A1B10F4A42F50E0B3
:1002A000BA2E8894AA1FAA2EA091A200A095AA22D5
:1002B000A50E58F0A091A100A21509F0AA95AA0ECA
:1002C000A093A10048F04A2D08C0A091A100BA1641
:1002D00008F0A395A093A1004FEF409364007F7BAB
:1002E000485F08F07064A0916000A395A09360003F
:1002F00051F0F894A9B7A160A9BF84FF02C0A0E49F
:10030000ABBF3FBE1895A0917400A395A093740055
:1003100041E050916800552329F085FF03C05A95AC
:1003200050936800A0919600A13018F02092990097
:100330000DC020929A002092A300A0919900AF5F77
:10034000A093990018F0AFEFA0939900F894A9B783
:10035000A160A9BF84FF02C0A0E4ABBF3FBE189557
:100360003FB64CB55DB58F7EABB7A074A21180616E
:10037000A0E0ABBFA9B7AE7FA9BF789481FD23C031
:10038000A2E096FDA3E0A5BF8260A0B396FDA09574
:10039000A2FF05C040936500509366003EC1A3E0F4
:1003A00096FDA2E0A5BFAA27A064AABF8D7F85FF06
:1003B00001C026C140E0A0B396FDA095A2FD20C1DA
:1003C000409396000FC1A3E096FDA2E0A5BF8D7FEC
:1003D00061FF71C0A2E096FDA3E0A5BFAA27A064BB
:1003E000AABF82604093910050939200A0908F002A
:1003F0004A19B09090005B09BB24A22C4C385205DE
:1004000018F42092950049C0A091D400AA2359F174
:10041000483C520528F4A0E1BA2EAAE0AA2E23C037
:100420004836A1E05A0728F4A8E0BA2EAFE0AA2E79
:100430001AC0403DA2E05A0728F4A4E0BA2EAEE16B
:10044000AA2E11C0403AA5E05A0728F4A2E0BA2E1D
:10045000ACE3AA2E08C04839A8E05A0720F4A1E06E
:10046000BA2EA8E7AA2EC42EA0919300CA1AD52EA0
:10047000A0919400DA0ADD202AF4AFEFC094D09462
:10048000CA1ADA0A20929500A8E0A210A0E0CA14C5
:10049000DA0618F4A1E0A0939500409393005093DE
:1004A0009400409191005091920040938F0050939E
:1004B000900042E097C0A09165004A1BA0916600A1
:1004C0005A0B94FD82C093FD80C092FD7CC086FFD4
:1004D00003C0D52EC42E0CC05695479591FD73C010
:1004E0005695479590FD6FC0D52EC42ED694C794CF
:1004F00061FD19C0AC2DAC51AD2DA24008F005C076
:10050000DD2089F4AC2DA85C70F4A0916700A39560
:10051000AA2311F0A0936700AA3008F471C02092BA
:10052000960081606DC0A0916700AA2319F0AA957A
:10053000A0936700A22C5091BA0097FD06C0A0902E
:10054000C800533011F4A090D000AAEFAA0EA22D3B
:10055000A21DCA18DA0A4FB74170533049F4442338
:1005600021F087FD05C0806803C087FF01C08F7739
:10057000442359F0533031F4AFEFC094D094CA1AE9
:10058000DA0A03C040E050E020C0533049F4CC0CFC
:10059000DD1CAAE0CA1AD20818F4A0E0CA2ED22C98
:1005A000AFEFCA16D20418F04FEF50E00EC0A09182
:1005B000AC00CA9E412D000C441F50E008F012C050
:1005C0004FEF50E00FC05695479594FF07C0552355
:1005D00009F04FEFA42FA6954A0F521D4F3F520529
:1005E00008F04FEF40939600816061FF09C0AFE1D2
:1005F000A095A923AB299A2F8F7DBB2009F4806297
:10060000A8E1A093680085FF03C0AAE0A09368005A
:1006100061FD03C085FD01C08F7E85FD03C0A6E09E
:10062000A0936900F894A9B7A160A9BF84FF02C094
:10063000A0E4ABBF3FBE189511E00AC013E008C0AC
:100640001AE006C01EE104C014E602C018EC00C0A7
:1006500005E1BB27BA95F1F70A95D9F71A95C1F7C5
:1006600008952AE338E709C020E33CE806C02AE2FF
:1006700034EB03C025E238EC00C0B091AD00BA9570
:1006800009F4089512E0BB27AD9ABA95F1F7AC9A38
:10069000BA95F1F7AC98BA95F1F7AD98BA95F1F72C
:1006A000123009F0979A123009F4959AB091AD0082
:1006B000BA95F1F7123009F09798123009F495982D
:1006C000B7E8BA95F1F71A95F1F6022FB22FBA955D
:1006D000F1F70A95D9F73A9581F6AD9A0895221B5C
:1006E00039E0001F3A9509F40895221F211B18F4E0
:1006F000210F8894F6CF0894F4CF622C722CB0E0CE
:100700008894B395221F331FE0F737952795889477
:10071000912E802E020B130B10F4192D082D10F4BE
:10072000889401C00894661C771CBA9571F7172D40
:10073000062D0895322D11232AF43A95009510952F
:10074000031B130BF894029F712C002D129F912C08
:10075000802C7894780C172D921C292DB4E06B2EE8
:100760002695179507956A94D9F7332321F00095BC
:100770001095031B130B08950091B4000430A1F1F0
:10078000B0919600B15008F010C0B0916100B093E4
:10079000630020927E0020927F00209280002092B1
:1007A0008100209282006F7D1FC06090B400606263
:1007B000B0916100B093620008E317EC20917A00D9
:1007C00030917B0036952795B62DBA9541F0369538
:1007D0002795B62DBA95BA9511F0369527958DDFE8
:1007E00000937E0010937F00089500917E00B091E9
:1007F00062000B1B10917F00120928F40038BFEF34
:100800001B0740F009C00F37120508F405C00FE7B9
:1008100010E002C000E81FEF0093830010938400F3
:10082000089500918300B09180000B0F1091840017
:10083000B09181001B1F20E03091840033230AF423
:100840002A95B09182002B1F1AF4203F40F00AC075
:100850002F3008F407C00FEF1FEF2FE003C000E0B8
:1008600010E020EF30916300B0919B003B1718F42B
:10087000323030F009C0B0918400BB235AF004C07C
:10088000B0918400BB2332F4009380001093810068
:100890002093820008952091D70000918300000FDB
:1008A00010918400111F46DF11232AF40038BFEF96
:1008B0001B0740F009C00F37120508F405C00FE709
:1008C00010E002C000E81FEF002352F0B091620078
:1008D000B01B0B2F18F0013008F00AC001E008C06F
:1008E00000950F5FB09162000B0F08F001C00FEF91
:1008F0000093850008952091D80000918100109107
:10090000820018DF11232AF40130BFEF1B0740F0EB
:1009100009C00F3F120508F405C00FEF10E002C038
:1009200001E01FEF112352F0B0918500B01B0B2F97
:1009300018F0013008F00AC001E008C000950F5F10
:10094000B09185000B0F08F001C00FEF009363001A
:1009500008950FEF71FD1EC0B091D300BB23D1F0FD
:10096000B0917B00BB23B1F00FEF10917B00B7DE9D
:10097000F894B091730072FDB5E00B9F112D002D1E
:100980007894112309F00FEFB0919E000B1710F42B
:1009900000919E0000939D00089500917A001091AF
:1009A0007B0000541140B0919D0010F4BA9501C035
:1009B000B39511F0B0939D00089500C00895209163
:1009C000B500B6B1B6FDFBCF04B115B1B6B1BF7776
:1009D000B6B9B091AA00B395B093AA00B83060F14F
:1009E0002092AA00B091D200BB2321F1112329F05B
:1009F000B091AB00BF3F61F009C0B091AB000B17E5
:100A000039F020F4BB2321F0BA9502C0B395E1F38D
:100A100000919B00B093AB00B33650F400ECBB35B3
:100A200038F400E8B33520F400E4BB3408F400E007
:100A300000939B007F7E089510919B00B0E11B0FF7
:100A400008F41FEF10939B00B091B400B43081F014
:100A500000919B00B0916300B01B10F40091630003
:100A6000B0919D000B1708F00B2F502E00936400DF
:100A7000B091AA00B73009F47061089502E3F894C8
:100A8000B091D9000B9F012D000C001F7894B091FC
:100A90009B000B1710F000919B00009361000093E6
:100AA0006300502E0093640000939E0008952092EE
:100AB0007A00B0EFB0937B000895F8940CB51DB5A3
:100AC00020917400789430917500609076000093C6
:100AD000750010937600031B160971FD03C077FDA6
:100AE00080C028C0709077002093770027092223C8
:100AF00019F00FEF1FEF0EC08090780090907900F2
:100B00003093780060927900009175001091760022
:100B10000819190920917A0030917B0036952795A4
:100B2000020F131F10F40FEF1FEF00937A001093C2
:100B30007B002BC020917A0030917B003901B4E01A
:100B40008B2EB2E09B2E343040F08A949A94383049
:100B500020F072FD02C08A949A94769467948A94E5
:100B6000E1F726193709992021F0169507959A94EF
:100B7000E1F7200F311F20937A0030937B0028F497
:100B80003FEF30937A0030937B00323008F4706886
:100B900071FF02C0B3E00DC0B091C40000917100BC
:100BA000023838F0B395003A08F0B395B63008F043
:100BB000B5E09B2EB4E08B2E10917B0000917A0063
:100BC00024E0169507952A95E1F70819120928F0EF
:100BD000B02FB250B12FB20910F402E010E098012A
:100BE00026C020917A0030917B0039017694679479
:100BF0006694669466942619320906950695200F28
:100C0000321D20937A0030937B00323008F07F77DA
:100C100004E0369527953695279526952695201B31
:100C200010F0223008F422E089019090C40060FDA9
:100C3000FECFE0908B00F0908C006160B9B7B0619E
:100C4000B9BF380177FD41C07694679400938B005B
:100C500010938C00B92DB330E1F0B0FD04C0060D47
:100C6000171D930106C0000F111F0250120922E048
:100C700030E0B92DB33068F020938D0030938E00B2
:100C800000938700109388006092890070928A0018
:100C90003AC000938D0010938E002093870030930C
:100CA00088006092890070928A0071FF0DC0BFE0D9
:100CB000B0938D0020928E00B093890020928A001C
:100CC000B0938B0020928C001EC0669400938B0022
:100CD000B92DB33091F0B0FD03C0060D262D03C031
:100CE000000F025022E0B92DB33038F020938D0070
:100CF000009387006092890006C000938D002093C6
:100D000087006092890000917C0002FD0350013051
:100D100029F495FD0AC0B0E0B7B909C0023019F452
:100D2000B7E0B7B904C095FDF6CFB6E0B7B900910A
:100D3000A200000F10F4BBE60B270093A20060FD99
:100D4000FECFB2E0B0936E006160B9B7B061B9BFD9
:100D5000B72FB670D1F020917A0030917B00369594
:100D600027953695279571FF02C0B0E43B0FF894A4
:100D70000CB51DB5020F131F1BBD0ABD6160B0E1AC
:100D8000B8BFB9B7B061B9BF7894089568602092D0
:100D90007D0020E066FD20E206C0686020927D00B4
:100DA00020E266FD20E001E011E077FD11C0B72FE1
:100DB000B67009F0677F14E100917B00069509F495
:100DC00003950F3008F00FE071FF02C004E114E159
:100DD00060FD0FC0B0917D00BB2359F071FF06C0CC
:100DE000B0916E00BA95B0936E0011F470624FC06E
:100DF000ABDFB0B7B77FB0BFB8B1B0B7B860B0BF06
:100E0000B0917D00B395B0937D00B8B177FD06C079
:100E1000B1E071FDB3E0BA95F1F7B8B1B072B217B5
:100E200009F02AC071FF05C00395011708F00A9563
:100E3000CFCF63FD05C00395011708F0B4CFC8CF2D
:100E4000677FF8943CB56DB470907A00B0917B00E8
:100E5000770CBB1F08F4BFEF770CBB1F08F4BFEF84
:100E6000370D6B1E6BBC3ABD6160B0E1B8BFB9B75E
:100E7000B061B9BF789497CFB0916D00B13008F4EC
:100E800092CF63FD90CF0A9509F0A2CF7F7D20918C
:100E90008D0030918E00F894B0E1B8BF0CB51DB54F
:100EA000020F131F1BBD0ABDE0908700F090880061
:100EB0006160B9B7B061B9BF7894B72FB67039F037
:100EC000B0916D0072FFB395B0936D0009C075FFCE
:100ED00007C066FD05C063FD03C0BF91BF91F8C4A4
:100EE000089500E063FF01C001E0F89410917100E3
:100EF000B7E01B9F212D102D7894200F2695179574
:100F0000269517952695179510937100183718F4A4
:100F1000B8E7B093710000917100B09172000B17A7
:100F200020F060619798AC98959860FDFECFE090B6
:100F30008900F0908A006160B9B7B061B9BF0895C7
:100F4000B2E095FD0AC0F894B0937C00AD9AAB98DE
:100F500062FF01C0959A7894F4C0F894B0937C0035
:100F6000AD9A949862FF01C0979A7894EAC0B3E072
:100F700082FF24C095FD11C002E0F894B0937C007C
:100F8000E1E8F0E00093B1009598949A62FF02C006
:100F9000AC9A01C0AD987894D4C002E0F894B093B4
:100FA0007C00E1E8F0E00093B1009798AB9A62FF13
:100FB00002C0AC9A01C0AD987894C3C095FD0BC037
:100FC000F894B0937C00EBE6F0E0959862FF01C0E6
:100FD000AC9A7894B6C0F894B0937C00EBE6F0E05D
:100FE000979862FF01C0AC9A7894ABC0B4E095FDCD
:100FF0000AC0F894B0937C00AB9A949862FF01C049
:10100000AC9A78949EC0F894B0937C00949AAB9874
:1010100062FF01C0AC9A789494C0B5E082FF24C00E
:1010200095FD11C001E0F894B0937C00E7E7F0E093
:101030000093B100AC98AD9A62FF02C0979A01C0CC
:10104000AB9878947EC004E0F894B0937C00EBE811
:10105000F0E00093B100AC98AD9A62FF02C0959A9F
:1010600001C0949878946DC095FD0BC0F894B0932E
:101070007C00E5E6F0E0AC9862FF01C0979A7894B6
:1010800060C0F894B0937C00E1E7F0E0AC9862FFB8
:1010900001C0959A789455C0B6E095FD0AC0F894C1
:1010A000B0937C00949AAD9862FF01C0979A7894AF
:1010B00048C0F894B0937C00AB9AAD9862FF01C031
:1010C000959A78943EC0B1E082FF24C095FD11C08E
:1010D00004E0F894B0937C00EBE8F0E00093B100FA
:1010E0009798AB9A62FF02C0959A01C09498789441
:1010F00028C001E0F894B0937C00E7E7F0E00093AB
:10110000B1009598949A62FF02C0979A01C0AB987B
:10111000789417C095FD0BC0F894B0937C00E1E77C
:10112000F0E0979862FF01C0959A78940AC0F8940D
:10113000B0937C00E5E6F0E0959862FF01C0979AD5
:1011400078946F7E089524E630E0F9012092B10092
:101150009798AC989598AB9AAD9A949A6B7F0895AE
:10116000A2EBB0E009E00D9309E00D9304E00D93CC
:101170000FEF0D9303E00D930FEF0D930BE00D9325
:1011800003E00D9301E00D9301E00D93AEEBB0E0B1
:1011900001E00D930FEF0D930D930D930D930D93B0
:1011A00003E00D930FEF0D930FEF0D930D9305E2F9
:1011B0000D9300ED0D9308E20D9300E50D9304E00F
:1011C0000D930FEF0D9302E00D9300E00D930AE7EE
:1011D0000D930FEF0D9300E00D9301E00D9300E0F0
:1011E0000D9303E00D9300E00D9308952091B90055
:1011F0008B7F233009F48460B091BA00B33019F0CA
:101200009F7DB1FD90629F7BB091BB00B1FD90646A
:10121000223011F0886001C0877F08950A95E00FA1
:10122000F21DB4910895ECE1F0E00091B200F6DF18
:10123000B093D700ECE1F0E00091B300EFDFB093A2
:10124000D800EAE2F0E00091B800E8DFB093D900FE
:101250000091B800023008F402E000937300B091EE
:10126000CE000FEFB23009F400EAB33009F402E81F
:1012700000937200E8E3F0E00091D500CFDFB09377
:10128000A000089508952091C8003091C900B09140
:10129000BA00B33009F43E5097FF02C020E03FEFA0
:1012A000B32FB21B6B2EB25810F4B2E86B2E00E0D5
:1012B0000395609EB12DBD57D8F30093AC000895FF
:1012C0009068E1DFBFD9BED920E030E0B0E16B2EFD
:1012D000B5D9B09196002B0F321D6A94C9F7B4E0CE
:1012E00036952795BA95E1F7822E9F77CCDF089542
:1012F000F894E3E0F0E0B9E0B7BFB491B078C1F39F
:10130000F894A895B1B5B861B1BDB0E0B1BDB4E095
:10131000BEBFBFE5BDBF17DFB0E0B8BBB0E1B7BB34
:10132000B8E2B5BBB8E3B4BBB0E1B2BBB0EBB1BBA4
:101330002224A0E0B0E02D92AA31E9F7A0E6B0E0C7
:101340000FEF2D920A95E9F7B1E0B093A20008DF04
:10135000F7D2B6B1B460B6B90091CA000093AD003F
:10136000B1E0B0936A00F89471D97BD96BD97CD97C
:1013700069D97DD967D9F8940AEF1AEFA0B396FD21
:10138000A095A2FF1FC01A95C9F70A95B1F7E0E032
:10139000FCE1B591B43E39F4B591B03E21F4B5917C
:1013A000BF3F09F40CC0E0E0F395F395B591B83F69
:1013B00049F4B591B43931F4B591BA3A19F4EE273C
:1013C000F695099413DF2FDF5DDF5DDF0091CA0022
:1013D0000093AD00B8DEB2E0B3BFB2E0BEBDB2E094
:1013E000B5BDB1E5B8BFB9BFB0B7B77FB0BFB8B191
:1013F000B0B7B860B0BF20D97894DFDA209270001F
:10140000B3E096FDB2E0B5BFB0E4BBBFBB27B064AC
:10141000BABF8D7F1BD9626033E02CE0B09195009C
:10142000BB2321F42CE03A9509F4A5CF0BD980FF1A
:10143000A2CF8E7FB0919600B23078F3B92FBF71F2
:101440000091980000939700B0939800B01729F787
:101450002A9521F76D7FB3E096FDB2E0B5BFBB27BB
:10146000B064BABF8D7FB091D400BB2321F48062F9
:10147000B92FB0709B2F8F7B20926700E5D885FF36
:1014800005C0B0916700BA3008F08064D7D802E098
:1014900085FF01C000E0B0919600B017B8F3F89452
:1014A000E0D8DFD8DED87894D1D820928600B091E9
:1014B000BA00B33009F47DC0C1D8B091BE00B130DC
:1014C00008F477C0B0916A00B13008F472C085FDAD
:1014D00018C0B0919600BF3F08F46BC0F894CAD80A
:1014E0007894B2D8B0919600B130C0F7F894B9D8DA
:1014F000A7D8B7D87894A8D8B0919600BF3FB0F3DA
:10150000E0C2B3E09B2E9068F894BDDE78949CD83E
:10151000F8949F77B8DE80909600B0919600BF3720
:10152000789408F44EC088D8F894A4D878949A9403
:1015300051F7C6DEB82DB093C90088D8F89494D27C
:101540007894BAE09B2E9068F8949DDE78947CD8CD
:10155000F8949F7798DE80909600B0919600BF3700
:10156000789478F769D8F8947CD86AD87AD878943F
:101570009A9449F7A5DEB82DBB5FB093C8000B2F36
:101580001091C900125810F0100B20F4B2E80B0FA4
:101590000093C9005BD8F89400D275D2789454D8DF
:1015A000F89471DE7894B0919600BF3F08F48FCF25
:1015B00088C200919600B09186000B1710F000933E
:1015C000860042D801E0B091BA00B35009F405E0BA
:1015D000B0919600B01708F06ACFF8944BD84AD86B
:1015E00049D8789433D820926A0020926B002092D8
:1015F0006C00B0916B00B395B0936B00BF3F71F579
:10160000B0916C00B395B0936C00B091CC0009E13F
:10161000BA9559F002E3BA9541F00DE7BA9529F071
:101620000AEFBA9511F020926C00B0916C00B017DF
:10163000A8F089DD01D8B0916C00BA95B0936C0028
:1016400020926B00B091CB00B093AD00F89412D80B
:101650007894B091CA00B093AD00F6D7F1D7B091AD
:101660006800BB2319F485FF01C085CE01E085FD2C
:1016700001C006E0B0919600B01708F4BACFB0915F
:10168000BA00B35009F0E0D7B0916800BB2309F469
:1016900072CEF89458DD2092610020926200209270
:1016A0006300522C209264002092A1007894B091A3
:1016B000B700BB0FB0939F0020927E0020927F0066
:1016C0002092800020928100209282002092AA0025
:1016D00060E070E020927100B8E0B093AA00706101
:1016E000ABD7B1E074FDB2E0B7B9B6B1B068B064E1
:1016F000B6B9B6B1B6FDFDCF04B115B1B6B1BF777D
:10170000B6B9112309F00FEF0093AB0058D9B8E038
:10171000B093AA0070616ADDF894BFEFB0939B00AC
:10172000ADD9B0916100B0939B00B0939C00B09391
:101730009D007894B1E0B0936100B09363005B2E9C
:10174000B0936400B093A400B0919A00B093A3004A
:10175000B091BA00B33019F49F7D87FD906271603B
:10176000726020926D0098DCAEDCA1D9A6D99FD919
:10177000A4D99DD912DB00D8B4DBE2DB9ED906DB0D
:1017800065FD33D877FFE5D877FD07D9AADBEFDB16
:1017900094D903DB65FD45D8A4DB28DC8ED9F6DAC5
:1017A00065FD79D89EDB39DC88D9F7DA65FDA3D8E9
:1017B00098DB72DC82D9EADAB1E074FDB2E0B7B945
:1017C000B6B1B068B064B6B98CDB7DDC76D9F7D839
:1017D00071FF24C0B0919E00B0939B00B0939C0019
:1017E000B0919A00B093A300B1E0B093A40018E1C7
:1017F0002CE0B0916D00B11758F07D7F746020939C
:101800006F00B0919E00B0939B00B0939D0006C006
:10181000B0919600B13008F0ADCF64C072FF15C032
:1018200066FD13C0B0916F00BA9519F47B7F7860A4
:10183000A1CFB0936F00B0919600B13008F09ACF6D
:10184000B091BA00B33009F04DC020927000B09151
:1018500099000AEF1091D600112309F003E0B017A8
:1018600008F040C085FF04C0B0916800BB23D1F1EF
:10187000B091BA00B33081F495FD03C087FD04C078
:101880000BC087FF01C008C066FD06C06064B09150
:101890009E00B0939B0083CF00EF66FF05C0B09120
:1018A0009E00B0939B0000E2B0917B00B01708F45B
:1018B00061CF66FF17C06F7B9F7D87FD906274606C
:1018C000B2E1B0936F00B0919E00B0939B0052CFF5
:1018D000B0917000B395B0937000B0919600BB23A7
:1018E00009F002C020927000F8942DDC8090B900BD
:1018F000B2E0B093B9007ADC8092B9002092610026
:101900002092620020926300522C20926400209268
:101910009F0060E070E0789497D615DC0091D600C7
:10192000002319F0979AAC9A959AB6B1B460B6B9FB
:1019300085FF05C0B0917000B43008F01CCD55CEC5
:10194000EDE0F0E023D0053509F01BC0EEE0F0E05B
:101950001DD00A3A09F015C03AE0A2EBB0E0E3E08E
:10196000F0E014D00D9331963A95D9F739E1AEEB0A
:10197000B0E0EFE0F0E00AD00D9331963A95D9F758
:1019800002C0EEDB0AD0E8E2F0E00895E199FECF74
:10199000EEBBFFBBE09A0DB308951ED03AE0A2EB78
:1019A000B0E0E3E0F0E00D910FD031963A95D9F731
:1019B00039E1AEEBB0E0EFE0F0E00D9105D031960B
:1019C0003A95D9F712D00895E199FECF0DBBEEBB41
:1019D000FFBBE29AE19A0895EDE0F0E00FEFF4DF4B
:1019E000EEE0F0E00FEFF0DF0895EDE0F0E005E568
:1019F000EBDFEEE0F0E00AEAE7DF08953091AE00B9
:101A00000091AF00313011F40093B200323011F484
:101A10000093B300333011F40093B400343011F468
:101A20000093B600353011F40093B800363011F44D
:101A30000093C400373011F40093B900383011F42A
:101A40000093D500393011F40093CE003A3011F4F0
:101A50000093BA003B3011F40093BB00089525E0D9
:101A6000F5D52A95E9F70895FCD5FED500D602D61E
:101A7000E7D5F7D5F9D5FBD5FDD5E2D5F2D5F4D527
:101A8000F6D5F8D50895F6D5F2D5EED5EAD5D8D560
:101A9000F1D5EDD5E9D5E5D5D3D5ECD5E8D5E4D567
:101AA000E0D508958090AE009090AF00DAD5D9D5FA
:101AB000D8D5C6D58A94D1F7DDD5C2D59A94E1F7A9
:101AC0000895F894D1DF7894CADFC9DFB1E0B0930C
:101AD000AE00B1E0B093AF002092B000F894E2DF26
:101AE0007894B5E06B2E70909600B0D5B0919600CA
:101AF0007B16C9F7B13018F0BF3F40F107C07EDF59
:101B0000F8944BDFB1DFB8E0B1BDA9DF6A9459F7B3
:101B1000B091B000B395B093B000B33008F4DECF0D
:101B20009EDFB091AF00B395B093AF00F894B09141
:101B3000AE00BA95EEE3F0E0EB0FF21D049178945D
:101B40000395B091AF00B01708F4C6CF88DF87DFE8
:101B5000B091AE00B395B093AE00B091AE00BC3082
:101B600008F4B7CFFDDAF89418DFB8E0B1BD77DF3D
:021B7000BFCBE9
:00000001FF
